:1000000009C021C020C01FC01EC01DC01CC01BC015
:1000100093C09EC011241FBECFE9CDBF10E0A0E663
:10002000B0E0E2EEF3E002C005900D92A637B10712
:10003000D9F710E0A6E7B0E001C01D92A737B107DD
:10004000E1F7CBD0CCC1DCCFE199FECF8EBB6DBB4D
:10005000F894E29AE19A78940895E199FECF8EBBE4
:10006000E09A8DB3089580E388BB16BE089580E8BA
:1000700086BD82E086BD0895F89416B81FBC13BEF5
:1000800083E085BD17BA18BA80E385BF88950895C7
:10009000813059F0813028F0823049F0833071F49A
:1000A00008C080E388BB85E507C080E303C088E320
:1000B00001C08AE388BB8FEF86BF0895DDDF089516
:1000C000EFEAF4E03197F1F700C000008150C1F78A
:1000D00008958FE390E4A7E081509040A040E1F7BD
:1000E00000C000000895852DD3DF01FF0DC0F1DFB2
:1000F000652DC09176008C2F8F5F8F718093760075
:10010000A3DF8C2F6FEFA0DFA82CB82C83E0D8DF03
:10011000EACF80917600A1DF909176008F3F31F495
:10012000903220F49F5F90937600F3CF903218F0D6
:100130001092760080E008951F920F920FB60F92F2
:1001400011240D7F22240F900FBE0F901F90189541
:100150001F920F920FB60F9211248F939F9385B128
:1001600000FF02C092E201C091E697B900FF0BC008
:100170009C2DCC2031F0950D891710F4939401C07B
:100180009924882E06C08D3710F4439401C044246E
:10019000382E81E08027082F90E1991518F090E41F
:1001A000941548F444249924952D9150592E9F3F3D
:1001B00011F4082F04609F918F910F900FBE0F9044
:1001C0001F90189550DF86E97BDF8AEA682E852D1F
:1001D000815093E0592E58220895F89400E08AEA5D
:1001E000D81609F402E05AEAD52EA8954424992499
:1001F0000E7F90E896BD81E086BD20E328BB2BE012
:1002000027BB98B994E194BB15BC91E697B997EADE
:1002100096B913B812BE16BE83BF83E88FBD80E2C5
:1002200085BF19BE1BBE7894A89588E181BD84E482
:1002300081BD8DE312DFC82F882369F401FF08C058
:100240006B2DBA1441F463508DE3FEDE15DF03C05D
:100250008DE36FEFF9DECC2ECF3F09F4CC248FE392
:10026000FCDE882369F48FE301FF07C0672DECDE15
:100270008BE360E0E9DE0D7F04C06FEFE5DE01C0D7
:10028000782E9FEF791611F47724739486B18864E1
:1002900086B901FF87C0822D222031F49AEA6916BF
:1002A00011F4662401C053948F5F282E843031F5F9
:1002B00089DF6624E32CC2E7D0E010E040E8F42EAA
:1002C000F6BE8BE4FDDE16BE84E6FADE8991E81602
:1002D00018F01F5F1530A1F784E6F2DE8DE3BDDE76
:1002E00081508E3F08F464C0BEDECAE084E1E8DEDF
:1002F00086B7809586BFC150C9F75AC0833019F4BC
:1003000061DF8BE307C08C3041F45CDF33E0532EB8
:10031000CC248DE360E098DE4BC0883089F452DF56
:100320008FE360E091DEA3DE77247394C7E076BEAE
:100330008DE7C6DE02FDA0DE770CC150C1F7F4CF19
:10034000863041F43FDF852DA3DE8DE7B9DE8BDEFD
:10035000C0DEF9CF853081F435DFC4E0852D98DE2D
:1003600085E0AEDE80DE82E3ABDEC150B9F788EC1B
:10037000A7DE8CE8A5DEF1CF8730D1F423DFC1E61C
:10038000D0E010E0FE01319780819ADE852D80DE7D
:10039000888196DE1E5F67DE2296123199F78FEF15
:1003A0008FDEEDCF2224B5DE582E8F3F09F4552481
:1003B00083E058228BE351DE8F3F31F001FF05C00F
:1003C0008BE36FEF41DE55248EDE2AEA622E76BE85
:1003D0004EDE889502FD50DE81E072DEFACFF894A1
:0203E000FFCF4D
:1003E200FF4B4B4B4B4BE1E14BE14BE1E14B4B4BB9
:0603F2004B4B98A0A4ABE8
:00000001FF
